:1000000002002C0207110000000000C28C02024D09
:100010000000000207F70000000000C28E02028309
:1000200000000032000000000000003275A80075DA
:1000300081D375D00078FF7600D8FC7580FF75906D
:10004000FF75A0FF75B0FF781079C377FF09D8FB63
:100050003110200618200509300116C2B3D2B28033
:100060001511F474FD912074FE91208019C2B2D252
:10007000B353B01F11E743B0E030000A30B2FD3097
:10008000B3FD7FAA713375360D7537407563017501
:100090003202D21E7589117588AA758CFC758A6921
:1000A000758DE3758B5A75B80ED2A9D2AB9000C985
:1000B000E493B4122620031C200608200505300016
:1000C00013D2AAD2AFD28CD28E12022E700D120B86
:1000D000930214D975B80BD2A880E853B01F11E76A
:1000E00043B0E011E780F47A0778617900D9FED84F
:1000F000FADAF622D3C2B39134D2B37881790020F0
:10010000B3080020B3F530B3FD22D9F3D8EF80E473
:1001100075260078FEE8428052807B32DBFE20B1FB
:1001200011D3E52613F526E823F8B4FEE84380FF53
:100130008003C380ED303002D229303102D22A3020
:100140003404D2028006E52654E07003D20022B4C3
:100150008003D20122B44003D20322B4C004D204EB
:1001600080EAB42003D20622B4A0E1D20522E5271A
:10017000B4032FE530B4032B9001C9752A00C023C6
:10018000C21BE4936017C082C083C0E0F530120B3D
:10019000F0D0E0120D21D083D082A380E5D023756A
:1001A000300022B40BFC9001AB80D0136B5D4B434D
:1001B00055542D4542352D33424E5B662E421E1E50
:1001C000636626635E66177400136B2B5D654535A9
:1001D000553C443D421E5E5E66423B4542435D35B2
:1001E0003D443C1C3D2D422B5D4B654D3D2D354224
:1001F0002445243D2D4B244255432B5B1755344257
:100200003D44552442552442435D3D421C42435DDA
:10021000353D443C1C3D2D4265355D2C4D2B3D420A
:10022000655C2D1C242D422B1C5C5C177400900116
:10023000C9C3E4F8E4936004A33880F730D70B20F7
:10024000D60820D205B80C02E42274FF22C0D0C028
:10025000E0C082C08375D00820031530050330B29A
:1002600011E531600415318007E5336003FF51F972
:1002700051DED083D082D0E0D0D0758CFC758A69F5
:10028000D28C32C0D0C0E075D018E535600215358B
:10029000E5646002156430050FE562600B1562E5E8
:1002A000627005D2B2020A3FD0E0D0D0758DE375FE
:1002B0008B5AD28E32201421FCC0E0C000C00178DD
:1002C0003AE670FDC2A978617928E6600D18E6D992
:1002D000FAD001D000D0E0D2A922ECF680F3E533C9
:1002E0007016E5616012F533786179607E29E7F672
:1002F00060061918DEF8760022200125200611205C
:10030000051271307028753100853338753300223D
:1003100071E9800F911BC311FB500A74F991208081
:10032000F371A960097531038533387533000022F4
:1003300020024A716E30B2217C09C2B3715D30B2C5
:100340001820E011C2B3715D13DCF3D2B3715DE428
:10035000D2B3D2B222D2B380ED74FF80F37806D844
:10036000FEC2B27811D8FED2B27807D8FE22EF7C56
:1003700008D30320E003DCFA22B3DCF622716E30EE
:10038000B2FD7C09C2B3716130B21820E011C2B372
:10039000716113DCF3D2B37161E4D2B3D2B222D271
:1003A000B380EDD2B3D2B280D420B202E422EFC245
:1003B000B200D2B3782ED8FE71DB7F0871E220E064
:1003C00016C2B37803D8FE71DB03DFF071E2C2B36B
:1003D0007803D8FED2B222D2B380E8D2B2781BD84A
:1003E000FE22C2B27808D8FE2220B002E422EF7CBE
:1003F0000830B0F820E014C2B39111D2B3911603C3
:10040000DCEFD2B300C2B300D2B322D2B3911180D9
:10041000EA00D2B2002200C2B20022EFB4FF01E42F
:10042000237F0820E70AD2B3913423DFF6D2B32228
:10043000C2B380F47808D8FEC2B27808D8FED2B22F
:100440007808D8FE22000043413F3D3B570051440D
:1004500042403E3C58000D562A3A0F2901005038C0
:100460002C1E100200004A1D2D1F11030000370032
:100470002E201204000000002F2113050000452B40
:100480003022140600004D393123150700460000C4
:100490003224160800004F53332517090000470087
:1004A0003426180A000048003527190B000049526D
:1004B00036281A0C00004E37371C1B0D00004C006C
:1004C0002B4B000E000000590079473727170756BD
:1004D000007A4F3F2F1F0F5E00551312140D0E08A8
:1004E0000072191A1C151600008411221B1D1E0013
:1004F000007E39212324260000776A2A2B2D25002F
:1005000000765332342C2E000074293133353600F6
:100510005F63003A3B3C3D006269714142433E00EB
:100520006D6C61494B4446006F75604A4C4D450007
:100530006E7D705952544E00677C7E7E5A5B55002A
:100540006573585C6B64665700000200435856544C
:1005500052504B001F595755535169005E3060632C
:1005600042FF45001E663120100100005D6232210D
:10057000110200005C673322120300005B4E34233B
:10058000130400005A2B3524140500002F40362593
:100590001506006F4C643726160700001D3C3827EF
:1005A000170800493D4F3928180900483E4D3A299F
:1005B000190A00703F0F612A1A0B00464A65004471
:1005C0001B0C00712E630D2D5F41000000001B64A9
:1005D000245D25532B4C231D2C2D2D5B3354344D82
:1005E0003D453565433B3B23442C3C5545344C4409
:1005F0004D3C5325543D552B5D355B33631B5C43AC
:100600006424655C6C6E757676756E6D6D631D6CBD
:10061000662E1E6D26752E6336653E34464B4E5C47
:10062000564C5E361B6C2454251D2B3C2C2B2D3B2D
:10063000342C3D4D35453B253C3D45354C2D4D2419
:10064000541C555D5D5B5B66635E5C1B6456654672
:100650006C4E7576761E6E266D3E1D644B551C6E77
:1006600066633E4C465C4E4B56345E651B5E2456BC
:1006700025462B2323662C1B2D1D3353341C3D5D37
:10068000355B3B553C2D45354C3D4D245333542C67
:10069000554D5D455B3C636C5C2B6454653B6C6EF7
:1006A000757676756E6D6D641D3E4B251C4E31352D
:1006B0004A7052707D53715A4B6B68476C784F6922
:1006C00049487562507260497D58517A324D744084
:1006D0004C73011C5A2A38117A1D1406050E0605A2
:1006E000040D0C04030C0B03830B0A02010A090717
:1006F000780F077B5D177614583977487E7179211A
:100700007B297C015A22141A1112613A5D727C73A2
:100710007CC0D0C0E0C082C08375D01020010C2006
:10072000031ED083D082D0E0D0D03279127EFF2059
:10073000B2F0DEFBD9F730B2FD7FAA71A9020A3F01
:1007400030B34CE5346014B4FF03020A3F85343300
:10075000B4AA0575340280037534FFE53360253093
:10076000B2FDC2B37A0879EA30B204D9FB80152011
:10077000B2FD20E004C2B38002D2B30330B2FDDA8E
:10078000E57533007A1FDAFED2B330B3FD8093E40F
:100790007A0830B2FD20B2FD30B30703D2E0DAF2BE
:1007A000800503C2E0DAEB03FAE5287015EAB4101D
:1007B000028005B413CE80057534AA80C77528FF62
:1007C00080C2752800EA20E71720E00820E1092010
:1007D000E20A80B0D2B780F4D2B680F3D2B580A45A
:1007E00020E00820E10920E20A8099C2B780F4C223
:1007F000B680F3C2B5808DC0D0C0E0C082C0837522
:10080000D010D2B278B8D8FE30B2FD30B302802713
:10081000E47A0811401151DAFAC2B21151D2B21180
:1008200051C2B21151D2B21151C2B3C2B21151D29E
:10083000B3D2B2F5341156D083D082D0E0D0D032CA
:10084000C2B2115130B304D2E08002C2E003D2B28E
:10085000227912D9FE22204869204969204A69205C
:100860004B69204C69204D69204E69204F69204614
:1008700069204769E53430E709648460057528001C
:10088000801220403120412820422820432B204440
:100890002B20452BE534B4C2037534F29008E0E513
:1008A000346067B4E206F475F003A473405C80F62C
:1008B000020AFB020B1B020A4B020AA9020ABE0231
:1008C0000AD20209970209B40209C7020A080209FA
:1008D000F402093F020956020964020971020984FF
:1008E000020A29020AF3020ACE020ABA020AA50281
:1008F0000B69020B63020B5D020B4F020A94020AA2
:1009000092020A8B020B17020A6D020A85020AF78D
:10091000020A85020A81020A470209930209B0020B
:1009200009C3020A04020A770209F002093A02091D
:100930005102095F02096D020980D24D020B7275E6
:100940002900E5346007C228F536020B72D22880F0
:10095000F7D24E020B72752900853437020B72D222
:100960004F020B72752900853463020B72D2466107
:1009700072752800E5346004C21A6172D21A61727D
:10098000D2476172752800E5346004D2126172C2E8
:10099000126172D2486172752900E53420E004C208
:1009A000338002D23320E104C2326172D2326172EA
:1009B000D2496172752900E5346004C21B6172D2AC
:1009C0001B6172D24A6172752900E534601C30E007
:1009D0000B20E110D22AC22CC22B6172C22CD22B66
:1009E000C22A6172C22BD22C80F6C22BC22C80F09C
:1009F000D24C6172752900E53420E004C22961728D
:100A0000D2296172D24B6172752900E534601620DB
:100A1000E00D20E106C21ED21F6172D21E80F8C214
:100A20001EC21F6172D21E80F8717278DAD8FE3051
:100A3000040D30B2FD30B3FD1200E779AA71747471
:100A40002CC0E0E4C0E032D2406172752800E53489
:100A500020E00ED2B520E10DD2B620E20CD2B76173
:100A600072C2B580F0C2B680F1C2B780F2717279FD
:100A7000AB717479836174717279017174793A61BF
:100A80007479EE617479FED2196174717271E5C284
:100A90000B22D20B7172120B9371E575320275360F
:100AA0000D75374022D243617251E25006C2E0D246
:100AB000E18004C2E4D2E5F66172D244617251E28F
:100AC0005006D2E0C2E180EFD2E4C2E580E9D2452F
:100AD000617251E25006D2E0D2E180DBD2E4D2E58D
:100AE00080D57528007880E534C313C0D028F8E697
:100AF000D0D022A9386174D2416172752800E534E2
:100B0000600EF53264016004C20E6172D20E617231
:100B10007172A932020B74D2426172752800E534F9
:100B200020E50820E612753720801020E60575378D
:100B300040800875377D800375375EE534541F208B
:100B4000E40504F5366172FDC2E4CD042D80F47134
:100B500072742278807943F608D9FC61E571727469
:100B60001180F07172743380EA7172E480E579FC6F
:100B7000800279FA78A5D8FE8933AF33120330703A
:100B8000F9753100201903853338C21975330030E7
:100B9000B3FD22900BA278807943E493F608A3D9A1
:100BA000F922000000033000022301101223012269
:100BB0002223022222230222222302222223012292
:100BC0002223022222230222222300202233112266
:100BD000203322322323032333333333333303309D
:100BE00023300000307839760008E8646170F8221C
:100BF00020060C20050C200E4C200009020C45029A
:100C00000CA3020CFB12106F121619121766703427
:100C1000E5326403600A12109170291213177024D0
:100C20001211A5701F12135D701A12145B70151249
:100C3000147470101216DA700B9004C8E5309360CB
:100C4000031202B52212161912176670F7121091CC
:100C500070F212135D70ED12145B70E81214747070
:100C6000E31216DA70DE200F2720030CE53064143F
:100C70006010E5306439600EE53064487012B2B53A
:100C80008006B2B78002B2B6D20F20380F20390CDE
:100C9000900445E5309360031202B522203AFC30FF
:100CA0003BEE221216191217667099121960709491
:100CB0001219C6708F1217D9708A12135D708512BF
:100CC000145B70DE12147470D91216DA70D4E53029
:100CD000B41410B2B7201004D210801AC21074BA23
:100CE0000202B5B43910B2B6201104D2118007C285
:100CF0001174C50202B59018BE809812161912140C
:100D00005B709F121474709A1216DA7095E530B405
:100D10002207B2B7B21130110590054B8193020E34
:100D200011D208E530B428028006C2146430600293
:100D3000C21320060C20050C200E57200009020DBE
:100D400092020DBD020DF812106F121619E53264F1
:100D500003600C121091703512131770308003204D
:100D60001D2B1211A5702612135D702112145B70D9
:100D70001C12147470171216DA70129004C8E53041
:100D800093600AFE74F01202B5EE1202B5C208C2F8
:100D90000F2212161912109170F312135D70EE12D9
:100DA000145B70E912147470E41216DA70DFE53027
:100DB0009004459360D744801202B580D012161972
:100DC00012196070C81219C670C31217D970BE12FA
:100DD000135D70B912145B70B412147470AF1216F4
:100DE000DA70AAE530B4140280A3B43902809E9070
:100DF00018BE93B4FFBE809512161912145B70F6DC
:100E000012147470F11216DA70ECE530B42202A1FB
:100E10008D90054B9360DFB4FF01E48097200BFDBC
:100E200012103F12100A200515120FE312101EE5D2
:100E3000277009E530B47F0420150322C215120E75
:100E40008C120EC8700B121712120FBB120FD47136
:100E5000F02212103F12100AC20D200516E527706D
:100E60000CE530B47F07B2153015028016120FE37F
:100E700012101E120E8A120EF17008120FBB120F02
:100E8000D4B121852A30120FE622D2092005209004
:100E90000EB67901E4936009B5300EE920090542E8
:100EA00027C20922F4522780F8C923C9A380E590FC
:100EB0000EBF790180DE136B1A2A227A000000131C
:100EC0006B4A72147A1A2A00302919200A16200552
:100ED0001B900FAB79017E04E493B53005E96224E1
:100EE0008002DE02E422C923C9A380EC900FAF8008
:100EF000E33029F020051C900FABA9247E04E49375
:100F0000B53006E920E04380DBDE028010C903C96A
:100F1000A380EB900FAF80E2900FB780062005F81A
:100F2000900FB3A9247E04E493B53021E930E40E98
:100F3000C2E403DEFD7E0403DEFDF52480A6D2E4D8
:100F400003DEFD7E0403DEFDF52474FF22DE0302D2
:100F50000F58C903C9A380CF302008C22078C5E646
:100F600054EFF6302116C22120050A20330778C736
:100F7000E679DF800578C5E679F759F630221FC299
:100F80002220051320330778C6E679DF800578C76D
:100F9000E679DF59F6800778CCE679DF80F53023F3
:100FA00008C22378C6E654DFF6C1E413221A001300
:100FB000144A1A6B7A2A006B7A722A200511200AC9
:100FC0000EE530B44A0920380720390475308022F4
:100FD0007530812220050B301208E530B4110375FD
:100FE000308222200A03203301229010007B05E486
:100FF0009365306005A3A3DBF622A3E493F53022CA
:101000001422221A1A142A7A7A2A200A03200D019D
:10101000229010187B0380D77F3848305028200A50
:10102000032032012290103B7B02E493653060057F
:10103000A3A3DBF622A3E493F530227B72727B201C
:101040002B0D202C11302A219005CE7921800C9077
:101050000610792880059006607927200A0BAE30AB
:10106000E4936E6005A3A3D9F722A393F5302290F1
:1010700004C8E530937880C313C0D028F8E6D0D0F8
:10108000C21CC21D50065403C442232254304223C2
:1010900022E530FE64506008EE647F60580211B1B2
:1010A000200831200A2E300018200E15203D0B207C
:1010B0003C089010E879080210CC9010F079058077
:1010C0000B203D13203C109010DE7906E4931202B1
:1010D000B5A3D9F874FF229010E4790480EEE11DE5
:1010E00045E19DC5E046E0C6E11477E1F014F077F4
:1010F000E07EE0F07E300859203A41203B3E203827
:1011000025203922203D1F203C1C30000E200E0BD4
:101110001212D3747C1202B50212EF12131274B7BA
:101120001202B50212F730000B200E081212D3740F
:101130007C0202B512131274B70202B530000D2002
:101140000E0A74F01202B574840202B574D402025D
:10115000B5203A41203B3E200A2520382220391F65
:10116000203D1C203C1930000E200E0B1212E11203
:101170001312747C0202B512130574370202B530E3
:10118000000B200E08121312747C0202B512131207
:1011900074370202B5300008200E0574840202B5CF
:1011A00074540202B5AE30BE40059006CF8017E4FD
:1011B000229006AE790CE4936E600BA3A3A3D9F63C
:1011C00002133D021283EE643160F8300004200EF9
:1011D00001A3A3200834200A0920380E2039213029
:1011E000B623121312E4930202B520390830B6F286
:1011F00012125980ED30B6EA12125912127580E2BD
:1012000030B6DF80F612124B80D820381E203930DD
:1012100030B63430000B200E081212D3E4930202D1
:10122000B5121312E49344800202B520390730B698
:10123000E25113801630B6DB511312124B021267C3
:1012400030B6D0511380205113800E300007200E8D
:10125000041212E1221212DA22300007200E0412C8
:1012600012EF221212F722300007200E041212E8A9
:101270002212130B22300007200E041212F3221246
:1012800012FE2220082420381620391A1213123098
:101290000008200E05744A0202B574350202B551E9
:1012A0004B20390280E6516780E230000D200E0AA3
:1012B0001212D3744A1202B5800812131274B512B6
:1012C00002B52038062039AD74FF2251592039A5C6
:1012D00074FF22711274F00202B57112742A0202B4
:1012E000B5711274120202B5711274590202B5512D
:1012F000D380F051D380F3711274AA0202B5711237
:1013000074B60202B5711251DC8007711274360294
:1013100002B574E00202B5AE309006DB791BE493AF
:101320006E6006A3A3D9F7E422A3E493FE20080489
:10133000EE0202B574F01202B5EE0202B59006D2CA
:101340007903E4936E6007A3A3A3D9F6E4223000E7
:1013500004200E01A3A320080221E24113E530FE80
:1013600090144C7903E4936E6009A3A3A3A3A3D9BB
:10137000F4E422A3E49330E702D20C200A172008F9
:1013800014300C0B20380E20390B1213FA80062073
:10139000384420394920054B30004B200E48A3E546
:1013A0003264026001A3E493FE30080574F0120277
:1013B000B5EE1202B5300811300C0820380B1214AB
:1013C00005800620380820395A74FFC20C221213F7
:1013D000FA20394F80F312140520390280B7121415
:1013E0002E80B2A3A3A3E493547FFE300807448069
:1013F0001202B580C0C20C0202B520051C300015D7
:10140000200E1241E320051630000C200E0974F066
:101410001202B541E341DC41F974600202B574E0A7
:101420000202B520051C300015200E1241EA2005ED
:101430001630000C200E0974F01202B541EA610D5D
:10144000610074610202B574E10202B5110D5555D7
:101450000080B341413881B4494939E530201B024D
:10146000E422FE90146A7902616553334141385B8E
:1014700034494939E530201A02E422FE9014837978
:1014800001616564A74C4C29EA24C3F8E6F47005B1
:1014900076FF0214A8FF1215BCF4FB7C08EF03FFD3
:1014A00020E706EB03FBDCF522EB03FB20E7F7EF7D
:1014B000547FFFEA541F2323232C14FDEF03DCFD8C
:1014C00023F4FF1214CF8D30C20A120E5280B9EAF3
:1014D00024C3F8EFF622021565752DFF12016E2068
:1014E000B402D20D300515E52754E0B4E0028007C0
:1014F000E52754D0B4D005C2B2756241E4FA9188B0
:101500001215BCFBF460CFEA24C3F8E6FF7C08EBBD
:1015100013FB5008EF13FFDCF6021567EF1350F6CC
:101520008C2B8A2E8C2C200A081215F6AC2B20D579
:1015300036EF54FEFFEA2323232C14FDECF52FEFA6
:1015400003DCFDFF91CFEAF52D8D2A8D3030030AA3
:10155000E530B439057535208003853735120E1D09
:1015600002156D80999188C30AEAB410F6852D2E74
:10157000E52E04603220282F200635200529300072
:1015800008E532B40303201C1EE535701A792FE7F5
:10159000792CF712160F20E012E533700AD20A12E6
:1015A0000E1D85363580C6C20A81DC85373581D966
:1015B000E530B4140280F0B439CF80EBC0D0C00263
:1015C000EAB408124380FFEA5407FA1215EE43A06A
:1015D000FF52A00215E350EC43A0FF1215EE43802A
:1015E000FF52807A32DAFEE590D002D0D0220A741F
:1015F000FFC333DAFD22C2D5856364D10F20D5083D
:1016000020E008E56470F42220E0F8B2D580E9AA71
:101610002EB1BCAC2C23DCFD22AE309016B2790C7E
:10162000E4936E6005A3A3D9F722A3E493F53020D9
:101630000831200A2D20051B300013200E10E53242
:10164000640360059016CE800D9016D28008901627
:10165000CA80039016D6E52354C023239360031257
:1016600002B522E52354C02323FE603930E1F33074
:10167000E038203CED20052830001B200E18E53214
:101680006403600D9016CE74F01202B5EE93020260
:10169000B59016D280F19016CAEE9344800202B53E
:1016A0009016D680F42038BA80CB2005C8203AB2F4
:1016B00080C31F06270E2F05370D3F04470C4F032D
:1016C000570B5F02670A6F07770F2A00381D120059
:1016D00011141200191160006463E530B43814204D
:1016E0000A2B200828203807203904B21B801EB29C
:1016F0001A801A20050AB43007200A11D213800D6F
:10170000B4280D200A07200804D214800074FF2298
:10171000E42230141B203819203916203A1D203BB2
:101720001A203C12203D0FE530B41714C21FD21E00
:1017300022C21EC21F22D21ED21F22D21FC21E22AE
:10174000B40606C22BC22C8011B40E07D22AC22CBA
:10175000C22B22B40507C22CD22BC22A22B40DD030
:10176000C22BD22C80F43013A7AE309017A8E4938C
:1017700060096E600DA3A3A3A380F3BE1792D228C5
:10178000808BA3E420381020390D203A12203B0F23
:1017900093F536C228E10DA393F537C228E10DA3D6
:1017A000A393F563C228E10D06FF19010E95200DE4
:1017B000057D26230D2A30390419354F0C0D406460
:1017C00003084B7A0B065E90020571A60A037DBCE6
:1017D0000702BCD20F01FFFF00E530FE90194179EE
:1017E00007E4936E6007A3A3A3D9F6E42230B61AE8
:1017F00020384F203964A3A3E493FE60EE20080450
:10180000EE0202B5EE44800202B520380520391AF6
:1018100080E574AA1202B574C51202B51217F674E7
:10182000451202B5742A1202B52274B61202B574BA
:10183000C51202B51217F674451202B574361202BB
:10184000B52274AA1202B574451202B51217F774C4
:10185000C51202B5742A1202B52274B61202B5740A
:10186000451202B51217F774C51202B5743612028A
:10187000B52274AA1202B574C51202B5EFFE121792
:10188000FD74451202B5742A1202B52274B6120212
:10189000B574C51202B5EFFE1217FD74451202B5FC
:1018A00074361202B52274AA1202B5EFFE1217FDA9
:1018B00080D474B61202B5EFFE1217FD80E2005715
:1018C00043413F3D3B5900514442403E3C5A000D8C
:1018D000002A3A0F29010050382C1E10020000FF88
:1018E0001D2D1F11030000FF382E201204000035AB
:1018F0004E2F211305000045003022140600004D34
:101900003931231507004629003224160800544FA8
:1019100053332517090051472B3426180A0049482C
:101920004A3527190B0058495236281A0C00524ED6
:10193000FFFF1C1B0D004F4C1D2B4B530E3700009F
:101940000019504A7C4B2B414D4E5947586148294C
:101950006A525552565370557D53784F60495851CD
:10196000E530FE9019567905E4936E6006A3A3D97D
:10197000F7E42230B60920383320393D0217F7202A
:10198000381020391A74C51202B51217F7744502BF
:1019900002B574C51202B51219AC74450202B574D1
:1019A000C51202B51219B974450202B574AA120221
:1019B000B51217F7742A0202B574B61202B51217DF
:1019C000F774360202B5E530FEB41603021A3CB4D1
:1019D0007B03021A42B43103021A48B42903021AE3
:1019E0002DB421030219FBB471030219FFB4720371
:1019F000021A2DB47303021A2DE4227E5380027E54
:101A00005530B613203816203913742A1202B51235
:101A100017FD74AA0202B52038062039030217FD0B
:101A200074C51202B51217FD74450202B5742A126C
:101A300002B57E091217FD74AA0202B57E507F48D6
:101A4000800A7E477F4B80047E357F3530B6092083
:101A5000381D20391C0217FD20381020390F74C59D
:101A60001202B51217FD74450202B50172018C0114
:101A7000A601B2000000000000000000000000000D
:101A80000000000000000000000000000000000056
:101A90000000000000000000000000000000000046
:101AA0000000000000000000000000000000000036
:101AB0000000000000000000000000000000000026
:00000001FF
